:10000000ADC1C4C1C3C1C2C1C1C1C0C1BFC1BEC1F4
:10001000BDC1BCC1BBC1BAC1B9C1B8C1556E697659
:10002000657273616C20524620506F7765726D6502
:1000300074657220202020444C354E4547202020F6
:100040000A004144432D72617776616C75652041E9
:100050004443312020414443322020242D2D2D20A3
:1000600020242D2D2D200A0044696F646520202056
:10007000202D2D2D203A78782E78782064422D205E
:100080006175746F202020204144432D0A004C6F7D
:1000900067416D702020202D2D2D203A78782E7804
:1000A000782064422D2066203D202D2D3030204DBB
:1000B000487A0A00546865726D6F2020202D2D2D1E
:1000C000203A78782E78782064422D207A65726FF5
:1000D0002D61646A3A202D2D0A002020426174743B
:1000E000657279202020202D2E2D20566F6C747380
:1000F00020205374617475733A202D6F6F2D0A00A0
:1001000020205741524E494E4720202020204F5654
:1001100045524C4F414420207265647563652070E0
:100120006F7765720A000F00110015001A001F009A
:1001300025002C0033003C004600530060006E0098
:1001400080009300AB00C400E000FE0021014C01E0
:100150007901AC01E90128027602C8022203870373
:10016000FFFF0A000C000F00110015001A0020000C
:10017000270030003C0049005B006F008800A500AC
:10018000C800F50026016001A701F5015602C00272
:100190003903C803FFFF27002A002D003100340077
:1001A000380041004B0055005F0069008500A20047
:1001B000BF00EC0019016601B3010102940227039C
:1001C000F203FFFFA100A300A600AA00AD00B1004A
:1001D000B600BB00C000C600CC00D100D700DD00D7
:1001E000E300E900EF00F500FB00020108010E0149
:1001F00015011B01220129012F0135013C0142019A
:1002000049014E0155015B01620168016E017401F3
:100210007A01810187018D0193019901A001A60155
:10022000AC01B201B801BF01C501CA01D001D701BB
:10023000DD01E301E901EF01F501FB010102060225
:100240000B020F02140217021B02FFFFAA00AE00EE
:10025000B200B600BB00C000C600CB00D100D70082
:10026000DD00E200E800EE00F400F9000001050105
:100270000B01100116011C01220127012C01320182
:1002800038013D01430148014E01530158015E010F
:10029000630169016F0175017A01800185018B019C
:1002A000910197019C01A201A801AE01B401B9011D
:1002B000BF01C501CB01D001D601DC01E201E8019B
:1002C000EE01F401F901000205020A020F02130215
:1002D0001702FFFFA600A900AD00B200B600BC00E7
:1002E000C200C800CE00D500DC00E200E900F0004A
:1002F000F700FE0006010D0114011B0122012A0175
:10030000310138013F0145014D0153015A0161019D
:1003100067016D0174017B01810188018F019501E5
:100320009C01A201A901B001B701BD01C401CA012C
:10033000D101D801DE01E501EB01F101F701FD0179
:1003400003020902100217021D0224022A023002CF
:10035000340238023A023C023F02FFFF11241FBE62
:1003600020E0A89521BD20E025BFE8ECFBE0A0E659
:10037000B0E003C0C89531960D92A636D9F7A6E62F
:10038000B0E001C01D92AD38E9F702C000C0189579
:10039000CFEDD0E0DEBFCDBF80E384BB87E088BB7C
:1003A00081E057D100D18FEF32D18FEF30D183E090
:1003B000809360004ED1F7D0809160008F5F809372
:1003C0006000873018F082E080936000A7D18091B0
:1003D000600099278430910521F481E0F9D002D2A0
:1003E000EACF853091050CF446C085309105F9F4CB
:1003F00081E0EED0D92FC82FF5D1C032D10581F0E0
:10040000A19738F48CE380938A008DE280938B006F
:10041000D2CF8DE280938A008EE380938B00CBCF86
:100420008FE680938A008BE680938B00C4CF06977B
:1004300009F0C1CF83E0CCD0D92FC82F82E0C133DF
:10044000D807A0F084E680938B0087E6809388002D
:1004500084E0D695C7958A95E1F780E090E020E0AA
:100460000A962F5FC817D907D8F764C082E7809330
:100470008B0080E7EBCF82309105D9F581E0A8D0E1
:10048000D92FC82F8C2F8F70D8D08093840044E050
:10049000D695C7954A95E1F78C2F8F70CED0809373
:1004A000830034E0D695C7953A95E1F78C2F8F708D
:1004B000C4D08093820082E08BD0D92FC82F8C2F9C
:1004C0008F70BBD080938A0024E0D695C7952A957B
:1004D000E1F78C2F8F70B1D08093890094E0D6958E
:1004E000C7959A95E1F78C2F8F70A7D080938800DD
:1004F00062CF039709F05FCF8091610069D0D92F57
:10050000C82F80916200882389F0C333D10518F485
:1005100082E080936100C95CD34018F081E0809351
:1005200061008091610054D0D92FC82F8C2F9D2F4E
:1005300059D141CFC81BD90B8C2F9D2F0A96215D15
:1005400020937500805D8093770035CFFFCF80E3E7
:1005500085BB80E185BB15BA0895982F20E09923CB
:1005600014F480E285BB85B3805F85BB85B3805181
:1005700085BB15BA990F2F5F283088F385B3805F4C
:1005800085BB85B3805185BB0895E1DF84E7E5DF56
:1005900080E8E3DF8CE0E1DF80E8DFDF80EADDDFB9
:1005A00080E4DBDF08950F931F93CF93EEDFC0E06D
:1005B00008E610E0F12FE02F81910E2F1F2F43D07E
:1005C000CCDFCF5FC432B0F3CF911F910F9108956C
:1005D0001F93CF93DF93982F86EE86B997B9C0E02B
:1005E000D0E010E084E09DD2181730F481E00FD005
:1005F000CC5FDA4F1F5FF6CF54E0D695C7955A957A
:10060000E1F78C2F9D2FDF91CF911F9108950F93CC
:100610001F93082F1DBC1CBC18B786E082D2182B74
:1006200018BF83E08EBD0BBD1ABC18B786E079D227
:100630001823D9F31F910F910895805D8A3308F034
:10064000895F99270895843209F482E080589927B8
:100650000895582F40E020E030E0852F992784301E
:10066000910509F44AC08530910524F58230910541
:10067000C1F08330910564F4019709F048C0F32F6D
:10068000E22FE859FF4FB32FA22FA45EBF4F3DC00A
:10069000F32FE22FE859FF4FB32FA22FA859BF4FD6
:1006A00034C0F32FE22FE859FF4FB32FA22FAE5BD8
:1006B000BF4F2BC086309105B9F0863091055CF0B4
:1006C000079729F5F32FE22FE859FF4FB32FA22FF9
:1006D000A050BF4F1AC0F32FE22FE859FF4FB32F9E
:1006E000A22FAC54BF4F11C0F32FE22FE859FF4F98
:1006F000B32FA22FA652BF4F08C0F32FE22FE85905
:10070000FF4FB32FA22FA257BF4F8C9180832F5F33
:100710003F4F4F5F443208F4A0CF089580916000AE
:1007200098DF41DF84E673DF0895282F392F809109
:1007300064008130F1F130936700209366008BE212
:1007400080937500332374F180E090E060E0281717
:10075000390734F088519C4F6F5F28173907D4F759
:100760006150281B390B28513C4F80E090E040E05D
:100770002817390734F08C599F4F4F5F28173907D6
:10078000D4F74150281B390B2C593F4F80E090E0A3
:1007900050E028173907A4F00A965F5F2817390739
:1007A000DCF70EC08DE280937500309521953F4FA8
:1007B000CBCF8091660090916700281B390BBFCF8B
:1007C000281B390B932F822F0A96605D6093760069
:1007D000405D40937700515D50937900805D809338
:1007E0007A000895BF92CF92DF92EF92FF920F931B
:1007F0001F93CF93DF93E82EF92E8091600029DFBD
:100800002BD180916000833009F4CFC080916000CB
:10081000843009F456C080916000853091F1BB208E
:1008200031F18FEF0F3F1807F9F00C1B1D0BEC1A7D
:10083000FD0AE4E6F0E09F2D8E2D6E2F7F2F89D1EB
:10084000712F602F98D1262F372FCB0CD11C9D2DC7
:100850008C2D6E2F7F2F7DD1280F391F24563040CD
:10086000932F822F62DFEEC087E0F3DEEBC08CE3D4
:10087000809374009D2D8C2D64E670E06AD155DF65
:10088000E1C0BB24CB2DDD27CC0FDD1F0C2F1D2F8E
:100890000A561E4F912F802F4ED1E816F90678F494
:1008A000CC24DD24912F802F46D1082F192FCC5630
:1008B000DE4F8C2F9D2F3FD1D92FC82FB0CFB394AF
:1008C000E1CF80916300882309F44DC080916300DB
:1008D000813039F180916300823009F09CCFBB24D4
:1008E000CB2DDD27CC0FDD1F0C2F1D2F0C521D4FE4
:1008F000912F802F20D1E816F90688F464ECC62EDB
:100900006FEFD62E912F802F16D1082F192FCE5290
:10091000DD4F8C2F9D2F0FD1D92FC82F7CCFB394B3
:10092000DFCFBB24CB2DDD27CC0FDD1F0C2F1D2FE0
:10093000045B1D4F912F802FFED0E816F90688F436
:1009400074ECC72E7FEFD72E912F802FF4D0082F75
:10095000192FC65BDD4F8C2F9D2FEDD0D92FC82FBF
:10096000B9CFB394DFCFB82ECB2DDD27CC0FDD1F51
:100970000C2F1D2F0C531E4F912F802FDCD0E8160B
:10098000F90688F4E4ECCE2EEFEFDE2E912F802FC7
:10099000D2D0082F192FCE53DE4F8C2F9D2FCBD0C6
:1009A000D92FC82F93CFB394DFCF809161008130CE
:1009B00039F180916100823009F028CFBB24CB2D22
:1009C000DD27CC0FDD1F0C2F1D2F0E591E4F912F31
:1009D000802FB1D0E816F90688F4F2EECF2EFFEFA3
:1009E000DF2E912F802FA7D0082F192FC05ADE4F4E
:1009F0008C2F9D2FA0D0D92FC82F08CFB394DFCF35
:100A0000BB24CB2DDD27CC0FDD1F0C2F1D2F0A5D46
:100A10001E4F912F802F8FD0E816F90688F4A2EF91
:100A2000CA2EAFEFDA2E912F802F85D0082F192FE5
:100A3000CC5DDE4F8C2F9D2F7ED0D92FC82FB9CF04
:100A4000B394DFCFDF91CF911F910F91FF90EF9083
:100A5000DF90CF90BF90089580916400882309F4BF
:100A600054C082E78093710085E6809372008CE623
:100A70008093730080E280937E00809160008330D9
:100A800019F180916000843009F04AC080916300C0
:100A900099278130910589F08230910554F4892B92
:100AA00009F03EC080E28093840085E38093850056
:100AB00037C00297A9F582E301C081E380938400E7
:100AC00083E3809385002CC080916200882391F09D
:100AD00081E68093800085E78093810084E780939E
:100AE00082008FE68093830080916100805D809317
:100AF0008B00C7CF8DE68093800081E680938100D4
:100B00008EE68093820080E2EDCF81E680937100D3
:100B100082E68093720083E7809373008DE6ABCF0B
:100B20000895282F81E090E002C0880F991F2A9530
:100B3000E2F799270895F92FE82F3196C895802D6F
:100B400031979927982F8827C895202D820F911DBE
:100B500008955527002480FF02C0060E571F660F18
:100B6000771F6115710521F096958795009799F784
:100B7000952F802D089597FB092E07260AD077FD23
:100B800004D00CD006D000201AF4709561957F4FE8
:100B90000895F6F7909581959F4F0895AA1BBB1B6A
:100BA00051E107C0AA1FBB1FA617B70710F0A61B6D
:100BB000B70B881F991F5A95A9F780959095682FB4
:080BC000792F8A2F9B2F089565
:060BC80001000100000025
:00000001FF
